:0230D800C1161F
:02249600AC0791
:1024980074562BF8E6FF74562CF8E6FB900259F0B8
:1024A800EFC39480500D9002587401F0C374809F5C
:1024B800F98009E4900258F0EF2480F9ED89F0A43E
:1024C800FF900254E5F0F0A3EFF0900258E0602886
:1024D800900254E0FF3395E0FEC3EB9FFFE49EFEBD
:1024E800900256F0A3EFF0C3EE64809480503AE473
:1024F800900256F0A3F08031900254E0FF3395E04B
:10250800FE74562CF8E6FD7C00EF2DFFEC3EFE90A5
:102518000256F0A3EFF0D394FFEE64809480400954
:10252800900256E4F0A374FFF0900256E0FCA3E09A
:10253800FDD394FFEC6480948040037FFF22AF05B5
:012548002270
:0223DF00A9054E
:1023E10074562BF8E6FE74562FF8E6FBEEC3947F85
:1023F10050097A01C3747F9EFE8006E4FA74812E2F
:10240100FEEEFD7C00AF017E0012157BEF7807CE5A
:10241100A2E713CE13D8F8FFEA601FEBC39FFDE4D8
:102421009EFC900252F0A3EDF0C3EC6480948050C6
:1024310029E4900252F0A3F08020EB2FFFE43EFE4E
:10244100900252F0A3EFF0D394FFEE6480948040A9
:1024510009900252E4F0A374FFF0900252E0FEA34F
:10246100E0FF7C007D6212157B900252EEF0A3EF3B
:10247100F0900252E0FEA3E0FF7D7F12158D9002E5
:1024810052EEF0A3EFF0E0241DF0900252E0340090
:04249100F0A3E0FFD5
:012495002224
:0729F500E527FD3395E0FC2E
:0429FC00ED2FFF229A
:102E650074562DF8E6900252F0122FF5EF2480FFEC
:102E7500900252E0FD7C00EF3395E0FE12157B7C5D
:062E8500047DB012158D62
:012E8B002224
:0730B7005355F8EF425522CA
:071A36007F01122FF58F1C48
:101A3D00C200C3E51C950DFEE49400900252F0A384
:101A4D00CEF0300D2E900252E0FEA3E0FFC3EE6407
:101A5D00809480500FE51670037516031516E51664
:101A6D007049802BD3EF9406EE648094804039C288
:101A7D000D802E900252E0FEA3E0FFD39400EE64A1
:101A8D00809480400FE5167003751603D5161C75EE
:101A9D001601800DC3EF94FAEE6480947F5009D245
:101AAD000D851C0DD2008003E4F516E5094508707F
:101ABD0054300051300408850D5912300B804630DA
:101ACD000D20E50D2406FFE433FED3E5599FEE64AA
:101ADD0080F874809840028010E559C3950D501E12
:101AED008017E559D3950D40051230758017E50D1A
:101AFD0024FAFFE559C39F50051230818007E4F5A4
:051B0D004FD21ED204BE
:071B12007F06122FF58F1C66
:101B1900C200C3E51C9511FEE49400900252F0A3A3
:101B2900CEF030112E900252E0FEA3E0FFC3EE6426
:101B3900809480500FE51A7003751A03151AE51A77
:101B49007049802BD3EF9406EE648094804039C2AB
:101B590011802E900252E0FEA3E0FFD39400EE64C0
:101B6900809480400FE51A7003751A03D51A1C7505
:101B79001A01800DC3EF94FAEE6480947F5009D264
:101B890011851C11D2008003E4F51AE50945087096
:101B99005430005130080885115D12300B804630F1
:101BA9001120E5112406FFE433FED3E55D9FEE64C1
:101BB90080F874809840028010E55DC39511501E2D
:101BC9008017E55DD3951140051230758017E51131
:101BD90024FAFFE55DC39F50051230818007E4F5C3
:051BE9004FD21ED208DE
:101BEE007F07122FF5AD077B077F031224968F50C8
:011BFE0022C4
:07191700E4FF122FF58F1C05
:10191E00C200C3E51C9512FEE49400900252F0A39F
:10192E00CEF030122E900252E0FEA3E0FFC3EE6422
:10193E00809480500FE51B7003751B03151BE51B70
:10194E007049802BD3EF9406EE648094804039C2A8
:10195E0012802E900252E0FEA3E0FFD39400EE64BC
:10196E00809480400FE51B7003751B03D51B1C75FF
:10197E001B01800DC3EF94FAEE6480947F5009D260
:10198E0012851C12D2008003E4F51BE50945087090
:10199E005430005130090885125E12300B804630EB
:1019AE001220E5122406FFE433FED3E55E9FEE64BB
:1019BE0080F874809840028010E55EC39512501E28
:1019CE008017E55ED3951240051230758017E5122B
:1019DE0024FAFFE55EC39F50051230818007E4F5BF
:0519EE004FD21ED209DA
:0D19F300E55EC313FFE545C3132FF5452244
:100A9A0012286390029D7405F0E5B05407F54E7F65
:100AAA00011230B77E807F008E2B8F2C8E288F29E3
:100ABA00E4FF122FF58F45EF90960093754C00F5E1
:100ACA004D25E0FFE54C33FE74002FF58274973E06
:100ADA00F583E493F54C740193F54D122FAE750826
:100AEA00007509C8121A3675F002E550A42400F5FB
:100AFA0082E5F03494F583E493F53C740193F53D73
:100B0A00121917122F95122EFCD2AF43E602D2CA3F
:100B1A0043C9049002A030A6057430F080037431F2
:100B2A00F0122989122680301E05C21E122989E573
:100B3A005520E3030210E9301703020E0F7F041257
:040B4A0030688F1C64
:100B4E00C200C3E51C950EFEE4940090024EF0A385
:100B5E00CEF0300E2E90024EE0FEA3E0FFC3EE6408
:100B6E00809480500FE51770037517031517E5175E
:100B7E007049802BD3EF9406EE648094804039C286
:100B8E000E802E90024EE0FEA3E0FFD39400EE64A2
:100B9E00809480400FE5177003751703D5171C75E9
:100BAE001701800DC3EF94FAEE6480947F5009D242
:100BBE000E851C0ED2008003E4F517E5094508707A
:100BCE0054300051300508850E5A12300B804630D5
:100BDE000E20E50E2406FFE433FED3E55A9FEE64A5
:100BEE0080F874809840028010E55AC3950E501E0E
:100BFE008017E55AD3950E40051230758017E50E15
:100C0E0024FAFFE55AC39F50051230818007E4F5A0
:050C1E004FD21ED205BB
:070C23007F051230688F1CF1
:100C2A00C200C3E51C950FFEE4940090024EF0A3A7
:100C3A00CEF0300F2E90024EE0FEA3E0FFC3EE642A
:100C4A00809480500FE51870037518031518E5187D
:100C5A007049802BD3EF9406EE648094804039C2A9
:100C6A000F802E90024EE0FEA3E0FFD39400EE64C4
:100C7A00809480400FE5187003751803D5181C7509
:100C8A001801800DC3EF94FAEE6480947F5009D264
:100C9A000F851C0FD2008003E4F518E5094508709A
:100CAA0054300051300608850F5B12300B804630F5
:100CBA000F20E50F2406FFE433FED3E55B9FEE64C5
:100CCA0080F874809840028010E55BC3950F501E2F
:100CDA008017E55BD3950F40051230758017E50F35
:100CEA0024FAFFE55BC39F50051230818007E4F5C3
:050CFA004FD21ED206DE
:100CFF007F07123068AD077B057F041223DF1229AF
:100D0F00F575F002EFA42400F582E5F03490F58339
:100D1F00E493F53E740193F53FD2177F06123068C6
:020D2F008F1C17
:100D3100C200C3E51C9510FEE4940090024EF0A39E
:100D4100CEF030102E90024EE0FEA3E0FFC3EE6421
:100D5100809480500FE51970037519031519E51971
:100D61007049802BD3EF9406EE648094804039C2A1
:100D710010802E90024EE0FEA3E0FFD39400EE64BB
:100D8100809480400FE5197003751903D5191C75FE
:100D91001901800DC3EF94FAEE6480947F5009D25B
:100DA10010851C10D2008003E4F519E5094508708F
:100DB1005430005130070885105C12300B804630EA
:100DC1001020E5102406FFE433FED3E55C9FEE64BA
:100DD10080F874809840028010E55CC39510501E25
:100DE1008017E55CD3951040051230758017E5102A
:100DF10024FAFFE55CC39F50051230818007E4F5BA
:050E01004FD21ED207D4
:100E06007D067F05122E658F273018030210DFE45A
:060E1600FF1230688F1C82
:100E1C00C200C3E51C950AFEE4940090024EF0A3B8
:100E2C00CEF0300A2E90024EE0FEA3E0FFC3EE643B
:100E3C00809480500FE51370037513031513E5139D
:100E4C007049802BD3EF9406EE648094804039C2B5
:100E5C000A802E90024EE0FEA3E0FFD39400EE64D5
:100E6C00809480400FE5137003751303D5131C7524
:100E7C001301800DC3EF94FAEE6480947F5009D275
:100E8C000A851C0AD2008003E4F513E509450870B5
:100E9C0054300051300108850A5612300B80463010
:100EAC000A20E50A2406FFE433FED3E5569FEE64E0
:100EBC0080F874809840028010E556C3950A501E45
:100ECC008017E556D3950A40051230758017E50A50
:100EDC0024FAFFE556C39F50051230818007E4F5D4
:050EEC004FD21ED201EF
:070EF1007F011230688F1C25
:100EF800C200C3E51C950BFEE4940090024EF0A3DB
:100F0800CEF0300B2E90024EE0FEA3E0FFC3EE645D
:100F1800809480500FE51470037514031514E514BC
:100F28007049802BD3EF9406EE648094804039C2D8
:100F38000B802E90024EE0FEA3E0FFD39400EE64F7
:100F4800809480400FE5147003751403D5141C7544
:100F58001401800DC3EF94FAEE6480947F5009D297
:100F68000B851C0BD2008003E4F514E509450870D5
:100F780054300051300208850B5712300B80463030
:100F88000B20E50B2406FFE433FED3E5579FEE6400
:100F980080F874809840028010E557C3950B501E66
:100FA8008017E557D3950B40051230758017E50B70
:100FB80024FAFFE557C39F50051230818007E4F5F6
:050FC8004FD21ED20211
:100FCD007F03123068AD077B01E4FF1223DFE52AB2
:100FDD001229F775F002EFA42400F582E5F03490A4
:100FED00F583E493F540740193F541D2187F021215
:040FFD0030688F1CAD
:10100100C200C3E51C950CFEE4940090024EF0A3CF
:10101100CEF0300C2E90024EE0FEA3E0FFC3EE6452
:10102100809480500FE51570037515031515E515AE
:101031007049802BD3EF9406EE648094804039C2CE
:101041000C802E90024EE0FEA3E0FFD39400EE64EC
:10105100809480400FE5157003751503D5151C7537
:101061001501800DC3EF94FAEE6480947F5009D28C
:101071000C851C0CD2008003E4F515E509450870C8
:1010810054300051300308850C5812300B80463023
:101091000C20E50C2406FFE433FED3E5589FEE64F3
:1010A10080F874809840028010E558C3950C501E5A
:1010B1008017E558D3950C40051230758017E50C63
:1010C10024FAFFE558C39F50051230818007E4F5EB
:0510D1004FD21ED20306
:1010D6007D027F04122E658F2AE4F52FF530F5A0E8
:0310E6000212985B
:0D10E900121A361219177F061230688F1C7C
:1010F600C200C3E51C9510FEE49400900250F0A3D4
:10110600CEF030102E900250E0FEA3E0FFC3EE6456
:10111600809480500FE51970037519031519E519A8
:101126007049802BD3EF9406EE648094804039C2D8
:1011360010802E900250E0FEA3E0FFD39400EE64F0
:10114600809480400FE5197003751903D5191C7535
:101156001901800DC3EF94FAEE6480947F5009D292
:1011660010851C10D2008003E4F519E509450870C6
:101176005430005130070885105C12300B80463021
:101186001020E5102406FFE433FED3E55C9FEE64F1
:1011960080F874809840028010E55CC39510501E5C
:1011A6008017E55CD3951040051230758017E51061
:1011B60024FAFFE55CC39F50051230818007E4F5F1
:0511C6004FD21ED2070C
:1011CB007D067F05122E658F27E55530E21075F0F1
:1011DB0002E545A42432F582E5F03497801AE54503
:1011EB0090960093753300F53425E0FFE53333FE1D
:1011FB0074002FF58274973EF583E493FF7401938B
:10120B0090024ECFF0A3EFF0C2A990024EE0F54C46
:10121B00A3E0F54D75F002E550A42400F582E5F04E
:10122B003494F583E493F53C740193F53DC3E53CAD
:10123B00648094804004D21B800DC21BC3E4953D97
:10124B00F53DE4953CF53C20171FAF511229F57580
:10125B00F002EFA42400F582E5F03492F583E493D9
:10126B00F53E740193F53FD21720181FAF52122988
:10127B00F575F002EFA42400F582E5F03492F583C6
:0D128B00E493F540740193F541D218D2A907
:10129800122DDEEF7003020B2E900297E06431608E
:1012A8000302135D9002A0E0FF900298E06F6003D4
:1012B80002135D900208E0FEA3E0FF900204E0FC48
:1012C800A3E0FDB507EDECB506E990020CE0FEA33E
:1012D800E0FFEDB507DDECB506D920C5D69002A034
:1012E800E0FF123036900208E0FEA3E0FF9002040F
:1012F800E0FCA3E0FDB507EDECB506E990020CE0D3
:10130800FEA3E0FFEDB507DDECB506D920C5D69004
:101318000299E0FFA3E0FDA3E0FBA3E0900255F0F3
:10132800121BFF900208E0FEA3E0FF900204E0FC1D
:10133800A3E0FDB507EDECB506E990020CE0FEA3CD
:10134800E0FFEDB507DDECB506D920C5D69002A0C3
:10135800E0FF123021900297E06432600302141318
:101368009002A0E0FF900298E06F600302141390CF
:101378000208E0FEA3E0FF900204E0FCA3E0FDB554
:1013880007EDECB506E990020CE0FEA3E0FFEDB531
:1013980007DDECB506D920C5D69002A0E0FF1230D3
:1013A80036900208E0FEA3E0FF900204E0FCA3E010
:1013B800FDB507EDECB506E990020CE0FEA3E0FFF1
:1013C800EDB507DDECB506D920C5D6900299E0FF4A
:1013D800A3E0FDA3E0FB121DAF900208E0FEA3E02E
:1013E800FF900204E0FCA3E0FDB507EDECB506E9CB
:1013F80090020CE0FEA3E0FFEDB507DDECB506D9E1
:1014080020C5D69002A0E0FF123021301C1C9002AB
:1014180097E014600D047012900298E0FF12305AA1
:101428008008900298E0FF123097900297E0FFB48E
:101438000B02D216EFB41407D21CD21612298990C7
:101448000297E064156003020B2EC21C1229890260
:021458000B2E59
:0628630075FFDE75FFADFC
:10286900E4900252F0A3F0900253E004F070069055
:102879000252E004F0900252E0B427EBA3E0B41056
:01288900E668
:10288A0075B217122E8C122F3E121A211230BE1256
:08289A00308D121A090228A278
:0A308D00759A07759D0475F803227B
:102E8C00E58954F04401F589D2A9D28C438E60D2E5
:102E9C00ADD2BD43E70443F70475CA1175CBFE757B
:062EAC00E41375E5FE22AF
:102F3E00E4F5A775B0FF75BDFCF5A57590FF75A4FA
:0E2F4E000D7580FF75A6FF75E10375E3402247
:101A210075AB1975AA8075BC3875E8C175D10B22E3
:0730BE0075D49C75D7942224
:102FF50075AC38EF2438F5AC75AA8075AA90E5AAAA
:0530050030E5FBAF9C6B
:01300A0022A3
:0D3068008FBB75E8D1E5E830E5FBAFBF2276
:10298900AF4F9002547480F0E55530E204EF4410E3
:10299900FFE55530E104EF4420FFE55530E004EF51
:1029A9004440FF301C04EF4480FFE55520E304EF69
:0529B9004401FF8F9BAB
:0129BE0022F6
:10268000E526605724FE604724FE6022240370453F
:10269000301611A21CB3921C301C04C220803312CD
:1026A0002FAE8031301C2E121A00C21C802712302F
:1026B0000BE55530E0047F028010E55530E1047FE2
:1026C000048007E55530E2057F011230B7800363CF
:0C26D000550812300B122989E4F526226F
:091A090043E60875D983D2DE2200
:031A1E0002221C85
:10221C00C0E0C0F0C083C082C0D075D000C000C088
:10222C0001C002C003C004C005C006C00720DF0304
:10223C000222E6E50945086008E509150970021552
:10224C0008E54445436011E54415447002154314F8
:10225C0045437004F54FD21EE5B05407F525654E85
:10226C00600CE525654EF531753B0385254EE53B48
:10227C006035153BE53B702FE53130E010E525204E
:10228C00E00B90029EE4F0A3744BF0D21DE53130CC
:10229C00E208E52520E203752604E53130E108E586
:1022AC002520E103752602301D2E90029FE024FFAD
:1022BC00F090029EE034FFF0E5B030E005752601A9
:1022CC00C21D90029EE07002A3E0700CC21D900231
:1022DC00A0E0FF7D02122F1EC2DFD007D006D00572
:1022EC00D004D003D002D001D000D0D0D082D08383
:0522FC00D0F0D0E0323B
:083097009002A5EFF0021A00FF
:0E305A009002A5EFF0122EFC122FC60229895B
:0C307500754F04D21E75430075446422A0
:0C308100754F02D21E7543007544642296
:03000000020A00F1
:03000300021A03DB
:03000B00021A06D0
:03001300021A09C5
:03001B00021A0CBA
:03002300021A0FAF
:03002B00021A12A4
:03003300021A1599
:03003B00021A188E
:03004300021A1B83
:03004B00021A1E78
:03005300021A216D
:03005B00021A2462
:03006300021A2757
:03006B00021A2A4C
:03007300021A2D41
:03007B00021A3036
:03008300021A332B
:03008B00021A3620
:03009300021A3915
:03009B00021A3C0A
:0300A300021A3FFF
:0300AB00021A42F4
:100A0000787FE4F6D8FD9000007F007E20E4F0A31C
:0A0A1000DFFCDEFA75815E020A5574
:08309F00002400300018000CB1
:031A120002295155
:10295100C0E0C082C083852982852883740193F5F4
:10296100D2E493F5D3A3A353830F438380858229B4
:10297100858328D083D082301709853FCAE53EF58B
:08298100CBC217C2CFD0E03237
:031A33000228DFA7
:1028DF00C0E0C082C083852C82852B83740193F561
:1028EF00D5E493F5D6A3A353830F43838085822C1E
:1028FF0085832BD083D0823018098541E4E540F5DC
:09290F00E5C21853C97FD0E03283
:031A0600021F0FAD
:101F0F00C0E0C0F0C083C082C0D075D000C000C098
:101F1F0001C002C003C004C005C006C007E55530AC
:101F2F00E303021FFC758CF2758AFB301B0EE53D37
:101F3F00253AF53AE53C3539F539800DC3E53A9543
:101F4F003DF53AE539953CF539E55530E111301F4E
:101F5F0004C21F800A5008753900753A00D21F530A
:101F6F0032C3E539C41313540325E0FFE433FE7481
:101F7F009F2FF58274303EF58374019342321227FE
:101F8F0085E55530E010E539900272F0F551F4F522
:101F9F00525332FC8034E5536006D553035332FE5F
:101FAF00E5546006D554035332FD301A1DC21AB2E0
:101FBF001930190C433201755305E52FF551800A7D
:101FCF00433202755405E52FF552900272E4F0D3B7
:101FDF00E53D9403E53C64809480400E301B05740E
:101FEF0004F080069002727402F08532A0D007D000
:101FFF0006D005D004D003D002D001D000D0D0D06D
:08200F0082D083D0F0D0E03252
:10278500C3E53A9530FFE539952FFED3EF954DEE2C
:10279500954C4037301B0EE54D2530F530E54C3571
:1027A5002FF52F800DC3E530954DF530E52F954C70
:1027B500F52FE55530E110301304C2138009500799
:0C27C500E4F52FF530D213D21A80B522B3
:108000008953AA7A83C6D9FAD4BBEB0EA37DD44A8E
:10801000B740CC0093CCD59CBBACBF9E6A3A93577B
:10802000756A8FCB6286B2AAA822BA346FA19ED994
:1080300081C39813630CA99695D1A131544786A5A5
:10804000727596BC7334CC95CA7DE3E69F52D2FB21
:10805000B8A2CFE299F6DDCFC5A5CB1276DEA0D9C6
:1080600083789E1270B1C065B51CC61C7A2BA7BD63
:1080700088BD9CE66580A97C93009B894BB07B11F1
:1080800063DE85275EAEB535B062C73A8047B1CAB8
:10809000958EAB3473FEB6E39E1FA3524F4579CE47
:1080A0005D6179554DB69F9196D1AABB620F933C05
:1080B000782790845D94A63F94A3A233577F8C17B2
:1080C0007A24A0AA7F62DB02DB27F6C9B46AEA42FF
:1080D000D211EB70B79AFD7EE752EEB09C5EC82BD2
:1080E000AC8DC8D59D11EE4EE478F6D6AC2CDAED09
:1080F000BD04D22B9BA8E06ECAA0D3BC845BB4168F
:108100009D22BE8C9816EE84E97BFFFFB89AE99019
:10811000CCA8E187A96CEB51D171D56D800FA92C4A
:108120008B3AA591783DC84CBDABCF9D84E6B3F4A6
:1081300096AFACCA7789BDD4A9CAB4E067A799B095
:108140008526A90D8520DE18DB90F485AF77E2A1A6
:10815000C7C4DE7CA802EB49D287D7588283ABD84C
:108160008DCDA7B879A4C8A1BC9CCCDD8028ACF18A
:108170008D26A07F6846AB6B94159BC04B07798416
:10818000616A81C95A63AFFBAA37C01B7831A8BDA9
:108190008B86A03067FCA9E2901D944E3F3F68C3D8
:1081A0004B516640399B8A7080A9938D49DA7A00D9
:1081B0005DE5753D414888F0765182DF372A6AC314
:1081C00057D37D5E5B1BB5C4B4F3CFA38C53C13EC4
:1081D000A821C0998BDDD0E0B9D5C0596D2F982A60
:1081E0007BBB97396AAEBB28B094C23876D9A4E974
:1081F00086559AD563B2A7DC91789A034A16794CD2
:1082000061D782C75BDEB1DEAC6DC28F7ACFAB7057
:108210008E3AA2D06A74AC1D920995D84053695029
:108220004B45658A382B88367D978F9344ED7412C1
:1082300056EC6D2D38197E976AC9762129315B8AF3
:1082400047566B9C4814A1779F62B8D17443A7F43A
:108250008DA5A4F16F12B2FA9AE0A0604C3E764F61
:10826000590573B6466F963F8B129C30505F7E1255
:108270005F3573823C4180646A1172C4231752A433
:108280003BA05D1836CF8D8988EA9FF7593A8AF569
:108290006EF184D24DD790F878727DE52A1954E2B8
:1082A00038B854F029977BB8734087723F107087B5
:1082B00055BE6E683BC684C07374815536F36BDD62
:1082C0005A3E811A6026BC1EBC99D895968ECCC0A9
:1082D000B4EACEA59B2BE16CCB9ED35B8168AD95B8
:1082E0009257AF01839FD53FCBCCDE8D9448C36DB1
:1082F000A5EABB76855ACA86B520BEA46FAB9FCED1
:108300008943AB16850ADBE2D743EE32A738D8980B
:10831000BC1CD16699B7DC07C293C6FB72099B935C
:108320007E0D98D16BE9BC65B22FC48F7A44A9BE8B
:108330008CE5A36C6E97B54EA1B0AD32606492D857
:108340007EB9A30B7F88D8EAD6CCF02BAB86DF1999
:10835000C4A5DBC4A5B2E960D105D63D81CDAB880B
:108360008DE2A8317A81C9E2BE3FCEE2828EAFB9FA
:0D837000904EA4066C2CAFAF98B7A0BF5084
:10837D00627F3A677B88346127B717B1AAC7E5805A
:10838D0051B131944EA94C716AB3A09A2C9EAC494F
:10839D00EB73BD569871D2457796958D17A04256C1
:1083AD00D687416B6A83054F52973A84DB91A84675
:1083BD00317A0667518D166B0CC5EDC552E0379DB0
:1083CD001CD239B94ED1F69D6AE29ACBBCD26B7FE5
:1083DD006BAA8F8E48A9EC7D86CE23C3B1D5778A43
:1083ED0037B86699EFAE8B7782BBC5A579AE1A5EAD
:1083FD00438D8C762A972B7051C660C0FCD72A8F7F
:10840D0074C01EA2EFB78C7F35C0E2A6D0AA9F55CF
:10841D001A7E1560077A474CE29CE6923EA43159CC
:10842D007F88986B6381954C7092DD7EFB8A3F3D12
:10843D00396F7A5B2F7F5B5BB7B4FEB2CCCC1B87F9
:10844D006DBAFDA08BB7B381AFC571AD2FB2855E8F
:10845D003A881F6AA9852C57B7A7569BF8ACE460DC
:10846D00E08E5E6F4B83614BE98FD3794581BD31D2
:10847D00D4612449E16B1A44919B099628ACF165AE
:10848D00F097667B1C90B659739C4B837B88A33405
:10849D008C5F0942925E7C32D384A57BDD8FBE4713
:1084AD000A782E5D12756842718B16797486FE3CC2
:1084BD004470D75EE085626415BFB2BFD3DB73999C
:1084CD0011CEE7B6B4D0129C3AE21DCBF1D34F805A
:1084DD00FDACCB912DAD7781B5D2F4C920DB819068
:1084ED00DABF9EA1B9B6E38066C52FAF67B88869BC
:1084FD002D98EE8200A3717D02D378CE76E5039D93
:10850D00A6CEA4B1C6C6AE8E9DD08BB6B6BABD658D
:10851D006A8E9270AC8B0F5DC7ADE3A34EB54E6AFC
:10852D00A499C07C8992B35D80A3DA8FE09B064D40
:10853D00DD7FF66B7C8F756B99C4A2C22CDB3396F5
:10854D0038C975AEABC5768F0FD26AB9BCBEA269FC
:10855D00E1934C75568F566158B06BA47CB4D468BA
:10856D00369516756288D350B293EF7CB28476330C
:10857D00D6626C4A6C6AE54399994B93A2A9A061A6
:10858D00D29278755D8A23520B940D7A657EB3294C
:10859D00C05362360D511A249275856BDD7EDF3521
:1085AD004B65904995610C2D3774FE627F6F2D23BD
:1085BD0099575344836A2F480EA2D8A229BCFB7940
:1085CD00CDAED995E0AE7A79E1BF06A81FAEC65BF8
:1085DD00C086DE6A93863559CEAA6C9FFCB1C566FE
:1085ED008B94C076518AF653F9984882098ABA3A23
:1085FD00F46A4F530174174D54A37B9E31B47A6CBA
:10860D00E19DA9809A95575D239EF4850788FE33D9
:10861D00A15CC63EE459502C1A7C4D71D683FB39B2
:10862D007E68CC4BCE62392D4D73F560506BD11FEA
:10863D000A518C3D8361F23E9398219635AFCD6BF7
:10864D006A9F4585209C9566E1AAF3930398AC44F7
:10865D00B56EF051D06CAC3F8F8F89848695D04A22
:10866D0029780659536DCB36B57B0264D96DB71E8B
:10867D00344DEC371258B53296897A85069C3D55A6
:10868D00AA87906BB781C14AF18E3D75E17B7E273C
:10869D00DC52D036D0533228027A4E71FF865C3EC2
:1086AD00236FC455256DF83B8084A47381818B376E
:1086BD00526C665AF181F5612BBD4BBDF0DA139802
:1086CD0036CE91B6E3D0C69D75E3DECE37D61D848A
:1086DD0052B0A79590B2628728D8EFCFA3E28C98BD
:0D86ED006DC7B9AA5DC0108A1BCF6DBA2DF4
:1086FA00C3D77504A54D8EE7B0E08AFAE1F7DD7DB0
:10870A00F491ADBCDF41C2E9D857A0CCE341C9F12D
:10871A00CE7D79AEA35B85F9A0DF741AC4B9BAA677
:10872A00CD2782FEB29A95E3AC8D77D9BEB1AB3331
:10873A00B6D66A299CBD88BEAD3189CEE34FE150D9
:10874A00FACEB648E9FACFA4E6E2B0EEF4BADC7C97
:10875A00E1D28D7FB75799CEB43986A6D622CA9B65
:10876A00DB598F22BC679D17B0EA792ABCC7A5E9F5
:10877A00AE0B5DC78CB8751295E36EEFC4F7BFA256
:10878A00D5F48E77BF6FA2A3B7B67FEBC237A8D94D
:10879A00AD6F58C282A9659880E754A0A5D29C689B
:1087AA00AFA5664C96CA7B0692B25F12A70B94BD20
:1087BA00A19B56348A1A77759D497B4FD63FD5B30C
:1087CA00F0A7AD99E2C4C9E7E29CAE1DF35ADC8872
:1087DA00E3439050BB7F9F43BAF28E96DF3ED4D6D6
:1087EA00E6A59B6FC9A7AB38BFDD88DCCD26B6E10D
:1087FA00BF8A6FB99F0987ADA8B481DFD7F3D29436
:10880A00E8C6A115D1C2B497C93790E2D292B8820C
:10881A00BC5366D08FCC71BF8BFF5E9BAE9EA3F616
:10882A00B5E86B349A4C7D1693455E1EA48890A3D6
:10883A009BE34ED981166CC690ED6D45C686C44E33
:10884A00DD9798E3CC6BB1F2C9129307D6C0BE7517
:10885A00C3C36F6F994A7BC9964368C3B857ACEED6
:10886A00BDCE71BE9F2F801094195C93A06F89D4DE
:10887A00923D424571865A347B5E54C4AB2CA63A6B
:10888A00BCF375E0A7448AE8A06F691AABDF92FCD3
:10889A00981043E46E4D51C16D9641D893948AB6AF
:1088AA009E8155B686C36B9083CE50BF994B8790F5
:1088BA0095024A2F7EA86C9692FE7197CD19CD1F0C
:1088CA00E8A3A625DBDFC38FDCD0A8DCEEA1D8574E
:1088DA00DF978D27B8D69D19B9448D62DE81D48D74
:1088EA00E6CD9C05CAA8ACA1C1AA8B0ACFB2B9C76A
:1088FA00C2C57346A2E48BD2AD1E868BDCDCD7B62A
:10890A00EE1DA69BD773BA6ECF3096F8D8C0BEC3F9
:10891A00C2A26D2796277819925364E2B4D5AA1792
:10892A00BBED7119A00A82A998A8634AA97995533F
:10893A00A04D52F884E5703E940A7001C8DDC63A2B
:10894A00DF1399E9CCF8B1FFC89B9206D531BC5424
:10895A00C10A6C199553772D90FD62CEB1B0A590DE
:10896A00B5B668E6959575AF88ED509993A47C33B2
:10897A0083C432F16153491F696441E49762918467
:10898A00A74E5F4A8FBC726B86FC4EAE907A769C7D
:10899A007AB3258A4EF5316A4C401F82703D665E75
:1089AA0079282F5D5F6A43365A7526686DF75B3FF3
:1089BA0067B51BE84F693C6061D33F789A099920F3
:1089CA00B3B87050A5238BEFA44F6F7CB4669D4457
:1089DA00A3B150707B535ECE7A344D929DF5934A83
:1089EA00A4D75961875B68B07D1A45E089F373792A
:1089FA007BEE2BEB5B0B4380645A3D5B93458DBE4C
:108A0A00A3CB5BF58C806F3583B64B448CD972AFA0
:108A1A00766920CF49B72B9845C81854684A5D969D
:108A2A006F7E24C353D5369A4CC7179F5E0A4A27CE
:108A3A00556B08673AAD26664A9826FC804D7E2417
:108A4A00977F52DF867D6C1B83544D629137790A7A
:108A5A007E772A44544236E55185242C73E968AA64
:0D8A6A0079B72DD45B753C8650C119705D45
:108A770081471C4FBE00002F7C186739CE13756ADB
:108A87001E656E7C6A359D67474B34610429F96D15
:108A97000A547459D705FB30B5147C30A4053B57ED
:108AA7004D4EC662E91A774BDF310849A316F25FCC
:108AB700DE4E835C5611E546C135145BE13AE0961C
:108AC700C99737B3257111A7358F51A8FF7578BBA3
:108AD700ABA5D0AD805B8087A16C5688F35D85AF71
:108AE70018A599B84E6DFC9D167F8695075EDFA386
:108AF700FF8E8D9806490179196283844B5E34B5E0
:108B070001B057C73B8036B18C9505AA44728BB428
:108B1700D19B539FB14AB6743556A6715F446E9484
:108B2700E18AA29CF852A4821565337BB246D38DA5
:108B37008279DB8554387E6AEA56C27B0D5782B04C
:108B4700DCAEB6C80C8360B6EC9C70B3887D6FC191
:108B570016A8B3ADE4596E832265767FBE5208A18D
:108B67006195B9A65559FC872067AF7B6243828719
:108B7700007002780527A256753EB15F6538538E9F
:108B87003E88CD9F03576A88466B5F805848728A34
:108B9700A5712C75A920E44AB22D8948C01C626DC5
:108BA7007D63FC77232DB45E1C424359DB26266E7A
:108BB7000C5BAA68751CFC50CF3E1863DB41CF9C49
:108BC700AE9C12B6F673D9A8F49009A8AF7422B96F
:108BD70051A273A9215621814464FD80A0543AA46F
:108BE700D89A66AC2C60ED8F1C70A585424E3A92E0
:108BF7007D7C3184D434FE64484CE76DEA47119D8F
:108C07002197BFADEF663B96E679BA8E5956049722
:108C1700B37DA481762BF354F136E6512923C7732C
:108C2700CD69297B1F30705F8D425C589223706934
:108C3700E15603614B1449468F3248567932DA8C34
:108C47002689F8A34C5EA3923877CB8EF958FA9C05
:108C5700C1848589E1359C5F8642165CA02F307EF2
:108C6700D6737E8471387365F846EC5B0923976782
:108C77008851025981099F38F721BB42FC1C7B723E
:108C8700FB6E2184F33DF96F78533668D8319E74B3
:108C97007F5BB860E80CDA37601AF236E50B465DA1
:108CA700215462684D1FA250D035BE4E1E1B316342
:108CB700E052485FDD152D49CB37DE5E6B3D2998C5
:108CC700D098FDB4A87251A832900AA97475A8BBB0
:108CD70096A575ACE05A9986746AE287385B82ACD0
:108CE700CDA306B5736AD999AA7BD191095A989FE2
:108CF7006F89B492E3439473635C837E0157A0AE9C
:108D070023A930BFCA787CA9888CB8A1AE69ACAB5F
:108D1700A991E295F840B369EA4C146685394D8903
:108D2700787EF3910246687593586C6EA539837FF8
:108D3700ED6C0277382A1F5C4947DF6BE9481DA1B4
:108D4700379ED2B7E972FFA64D8B94A2706C1BAF0A
:108D57008796EA9BE1473270AE52CB6CDD3EF18ECF
:108D670016823992A246167309536866EB2EDD7296
:108D77002D5B0262D9124B40F429084994225B7893
:108D870020728A889C40E1719B5494696E316A73A2
:108D97007F59EB5E4D096E332415E4310504925576
:108DA7009A4C065F1D159E45F72A11419D0DDD550D
:108DB700B9434F50130495386325AA4B6B295F8439
:108DC7004083A69E8E5B76909877B590655BE2A10F
:108DD7001E8A4D910A3E1B694F4D1C68D43C848DF9
:0D8DE7003982E094C0499D77E959926E4EA3
:108DF40037687BCE65A76E701EC14E3436FE582C84
:108E0400318187C0828D98EF516E824E65577A2DDD
:108E1400421183FB6A276E3618F2423024663EEC18
:108E240011CE621B57BD69FB1F974EFE321A489E36
:108E340013CC5A8D4701529C05EF388B249C49254D
:108E440025E07F877DB69768531F87146D09849941
:108E54004EFF932C7B56811A2D3E57933A8E55859F
:108E6400288378986DB07F143389618142EA577CF6
:108E7400208264EA4EDD57D6086F3842218443428B
:108E84001D4074406FE7873A40C372C557086D2F81
:108E9400367A79E261A3675B13D63EE623033F810A
:108EA400146E66D65EA5731E2B025CBF423D5B2E1C
:108EB40028D27213610D6F3425195A4A48F1701281
:108EC4004F66ABA3AC65C8A686E6BD5EA5CEBFCF94
:108ED4008C9BD322BD99C59C73EFA0628569A2596E
:108EE400773CC921BFF3D2FA88FAB8649B26B0F75D
:108EF4007B20C090AB6FB537668296EA80A3A2BA96
:108F04007CF2D40ECFB2E6E4A02ED1D2B599CB2612
:108F140093BAD64DBD1BC1C66D1796E2799F94A432
:108F240067FFB8BCAEC8C169775FA71A8A82A14B34
:108F34006CB6B3ADA04FAC115F8392377E57A2E9F4
:108F44007FA5D946D767F104AC9EE06FC639DD979B
:108F5400A7C2EBAED390D90584D2AECA9160ABEB75
:108F64007E78CE14C2ADD38B8773B4D895A8A99B51
:108F740071FBB5B89EF9A73B571886296EA38F9449
:108F840068BFBEE8B9B3D02588C9B9E09D34B268DA
:108F94007ABCBD29A3EBA8A154157E1C612B7C9A35
:108FA4005074A1C6987CABDA62A1933F779B8F681B
:108FB4005BE7A40191D49ED2538C8792750D9B02DA
:108FC4007928D438D3CDEEE1ABF4E13FC882E1583F
:108FD400ACF9F256DBA5E2818FAEBAFD9EE2BAB1DE
:108FE4008E76DF3ED4F6E6E69BD0CA28ABDAC09F85
:108FF40089BFCE2AB805C0CE711EA08EFC1CFC1FF2
:10900400FC23FC26FC2AFC2DFC31FC34FC38FC3B04
:10901400FC3FFC42FC46FC49FC4DFC50FC53FC5715
:10902400FC5AFC5EFC61FC64FC68FC6BFC6EFC722C
:10903400FC75FC78FC7BFC7FFC82FC85FC88FC8B4B
:10904400FC8FFC92FC95FC98FC9BFC9EFCA2FCA56E
:10905400FCA8FCABFCAEFCB1FCB4FCB7FCBAFCBD98
:10906400FCC0FCC3FCC6FCC9FCCCFCCFFCD2FCD5C8
:10907400FCD8FCDBFCDEFCE0FCE3FCE6FCE9FCECFD
:10908400FCEFFCF2FCF4FCF7FCFAFCFDFD00FD0235
:10909400FD05FD08FD0BFD0DFD10FD13FD15FD186F
:1090A400FD1BFD1EFD20FD23FD25FD28FD2BFD2DB3
:1090B400FD30FD33FD35FD38FD3AFD3DFD3FFD42FC
:1090C400FD44FD47FD49FD4CFD4EFD51FD53FD564C
:1090D400FD58FD5BFD5DFD60FD62FD65FD67FD699D
:1090E400FD6CFD6EFD70FD73FD75FD78FD7AFD7CF4
:1090F400FD7FFD81FD83FD85FD88FD8AFD8CFD8F4F
:10910400FD91FD93FD95FD97FD9AFD9CFD9EFDA0AF
:10911400FDA3FDA5FDA7FDA9FDABFDADFDAFFDB212
:10912400FDB4FDB6FDB8FDBAFDBCFDBEFDC0FDC27B
:10913400FDC4FDC7FDC9FDCBFDCDFDCFFDD1FDD3E4
:10914400FDD5FDD7FDD9FDDBFDDDFDDFFDE1FDE353
:10915400FDE5FDE7FDE8FDEAFDECFDEEFDF0FDF2C9
:0D916400FDF4FDF6FDF8FDFAFDFBFDFDFD3F
:10917100FFFE01FE03FE05FE07FE08FE0AFE0CFED1
:109181000EFE10FE11FE13FE15FE17FE18FE1AFE4E
:109191001CFE1EFE1FFE21FE23FE25FE26FE28FECE
:1091A1002AFE2BFE2DFE2FFE30FE32FE34FE35FE52
:1091B10037FE39FE3AFE3CFE3EFE3FFE41FE43FED7
:1091C10044FE46FE47FE49FE4AFE4CFE4EFE4FFE61
:1091D10051FE52FE54FE55FE57FE58FE5AFE5CFEED
:1091E1005DFE5FFE60FE62FE63FE65FE66FE67FE7B
:1091F10069FE6AFE6CFE6DFE6FFE70FE72FE73FC10
:1092010088FC8BFC8DFC8FFC92FC94FC97FC99FCF8
:109211009BFC9EFCA0FCA2FCA5FCA7FCA9FCACFC51
:10922100AEFCB0FCB2FCB5FCB7FCB9FCBCFCBEFCAE
:10923100C0FCC2FCC5FCC7FCC9FCCBFCCDFCD0FC0E
:10924100D2FCD4FCD6FCD8FCDBFCDDFCDFFCE1FC71
:10925100E3FCE5FCE8FCEAFCECFCEEFCF0FCF2FCD7
:10926100F4FCF7FCF9FCFBFCFDFCFFFD01FD03FD3B
:1092710005FD07FD09FD0BFD0DFD0FFD11FD13FDA5
:1092810015FD17FD19FD1CFD1EFD20FD21FD23FD12
:1092910025FD27FD29FD2BFD2DFD2FFD31FD33FD85
:1092A10035FD37FD39FD3BFD3DFD3FFD41FD43FDF5
:1092B10044FD46FD48FD4AFD4CFD4EFD50FD52FD6D
:1092C10053FD55FD57FD59FD5BFD5DFD5EFD60FDE7
:1092D10062FD64FD66FD68FD69FD6BFD6DFD6FFD61
:1092E10070FD72FD74FD76FD78FD79FD7BFD7DFDE0
:1092F1007EFD80FD82FD84FD85FD87FD89FD8BFD61
:109301008CFD8EFD90FD91FD93FD95FD96FD98FDE3
:109311009AFD9BFD9DFD9FFDA0FDA2FDA4FDA5FD68
:10932100A7FDA8FDAAFDACFDADFDAFFDB1FDB2FDF0
:10933100B4FDB5FDB7FDB8FDBAFDBCFDBDFDBFFD7A
:10934100C0FDC2FDC3FDC5FDC7FDC8FDCAFDCBFD06
:10935100CDFDCEFDD0FDD1FDD3FDD4FDD6FDD7FD94
:10936100D9FDDAFDDCFDDDFDDFFDE0FDE2FDE3FD24
:10937100E5FDE6FDE7FDE9FDEAFDECFDEDFDEFFDB7
:10938100F0FDF2FDF3FDF4FDF6FDF7FDF9FDFAFD4B
:10939100FBFDFDFDFEFE00FE01FE02FE04FE05FEDC
:1093A10007FE08FE09FE0BFE0CFE0DFE0FFE10FE71
:1093B10011FE13FE14FE15FE17FE18FE19FE1BFE0C
:1093C1001CFE1DFE1FFE20FE21FE22FE24FE25FEA8
:1093D10026FE28FE29FE2AFE2BFE2DFE2EFE2FFE46
:1093E10030FE32FE33FE34FE35FE37FE38FE39FEE6
:1093F1003AFE3CFE3DFE3EFE3FFE40FE42FE43FE87
:10940100B1FEB4FEB7FEB9FEBCFEBFFEC1FEC4FE96
:10941100C6FEC9FECCFECEFED1FED4FED6FED9FEDE
:10942100DBFEDEFEE1FEE3FEE6FEE9FEEBFEEEFE26
:10943100F0FEF3FEF6FEF8FEFBFEFDFF00FF03FF6C
:1094410005FF08FF0BFF0DFF10FF12FF15FF18FFAF
:109451001AFF1DFF20FF22FF25FF27FF2AFF2DFFF7
:109461002FFF32FF35FF37FF3AFF3CFF3FFF42FF3F
:1094710044FF47FF49FF4CFF4FFF51FF54FF57FF88
:1094810059FF5CFF5EFF61FF64FF66FF69FF6CFFD0
:109491006EFF71FF73FF76FF79FF7BFF7EFF81FF18
:1094A10083FF86FF88FF8BFF8EFF90FF93FF96FF60
:1094B10098FF9BFF9DFFA0FFA3FFA5FFA8FFAAFFA9
:1094C100ADFFB0FFB2FFB5FFB8FFBAFFBDFFBFFFF1
:1094D100C2FFC5FFC7FFCAFFCDFFCFFFD2FFD4FF39
:0D94E100D7FFDAFFDCFFDFFFE2FFE4FFE76B
:1094EE00FFE9FFECFFEFFFF1FFF4FFF7FFF9FFFCE1
:1094FE00FFFE0000000300050008000A000D00102A
:10950E00001200150018001A001D001F0022002571
:10951E000027002A002D002F003200340037003AB9
:10952E00003C003F0042004400470049004C004F01
:10953E000051005400570059005C005E0061006449
:10954E0000660069006B006E007100730076007992
:10955E00007B007E0080008300860088008B008EDA
:10956E000090009300950098009B009D00A000A322
:10957E0000A500A800AA00AD00B000B200B500B86A
:10958E0000BA00BD00BF00C200C500C700CA00CCB3
:10959E0000CF00D200D400D700DA00DC00DF00E1FB
:1095AE0000E400E700E900EC00EF00F100F400F643
:1095BE0000F900FC00FE0101010401060109010B86
:1095CE00010E0111011301160118011B011E0120CC
:1095DE00012301260128012B012D01300133013514
:1095EE000138013B013D0140014201450148014A5C
:1095FE00014D0202040404040404040404040404DB
:10960E000404040404040404040406060606060600
:10961E0006060606060606060606060606060606DC
:10962E0006060606060606060606060606060606CC
:10963E0006060606060606080808080808080808AA
:10964E00080808080808080808080808080808088C
:10965E000808080A0A0A0A0A0A0A0A0A0A0A0A0A62
:10966E000A0A0A0A0A0A0A0A0A0A0A0A0A0A0A0A4C
:10967E000A0A0A0A0A0A0A0A0C0C0C0C0C0C0C0C2C
:10968E000C0C0C0C0C0C0C0C0C0C0C0C0C0C0C0C0C
:10969E000C0C0C0C0C0C0C0C0E0E0E0E0E0E0E0EEC
:1096AE000E0E0E0E0E0E0E0E0E0E0E0E0E0E0E0ECC
:1096BE000E0E0E0E0E0E0E0E0E0E0E0E0E0E0E0EBC
:1096CE00101010101010101010101010101010108C
:1096DE00101010101010101010101010101010127A
:1096EE001212121212121212121212121212151546
:1096FE0015180000000080005556400033342AAB88
:10970E00249320001C72199A1746155613B2124A4A
:10971E00111210000F100E390D7A0CCD0C310BA357
:10972E000B220AAB80008000800080008000800049
:10973E00800080008000800080008000800080001B
:10974E007AAB75C3713B6D096925658462225EF83B
:10975E005C0059365697541D51C74F914D794B7D2C
:10976E00499A47CE4618447742E9416C40003EA3E1
:10977E003D553C153AE139BA389E378C36853587DA
:10978E00349233A632C231E6311130432F7C2EBBD8
:10979E002E002D4B2C9B2BF12B4B2AAB2A0F29770E
:1097AE0028E4285427C9274126BD263C25BE25443A
:1097BE0024CD245823E72378230C22A3223C21D73F
:1097CE002174211420B6205A20001FA81F521EFDFE
:1097DE001EAB1E5A1E0A1DBD1D711D261CDD1C95BD
:1097EE001C4F1C0A1BC61B841B421B021AC31A8663
:1097FE001A491A0E19D3199A1961192A18F318BD94
:10980E0018891855182217EF17BE178D175D172ECA
:10981E00170016D216A51679164E162315F815CF63
:10982E0015A6157D1555152E150714E114BB1496A6
:10983E001472144E142A140713E413C213A0137FC8
:10984E00135E133E131E12FE12DF12C012A21284FA
:0D985E0012661249122C121011F411D811CB
:10986B00BC11A11186116C11511137111E1104106D
:10987B00EB10D310BA10A2108A1072105B104410A8
:10988B002D101610000FEA0FD40FBE0FA90F940F57
:10989B007F0F6A0F550F410F2D0F190F050EF20E8B
:1098AB00DE0ECB0EB80EA60E930E810E6E0E5C0E58
:1098BB004B0E390E1F0E050DEB0DD20DBA0DA10D72
:1098CB00890D710D5A0D430D2C0D160CFF0CEA0C66
:1098DB00D40CBF0CAA0C950C800C6C0C580C440CC3
:1098EB00310C1D0C0A0BF80BE50BD30BC10BAF0B9B
:1098FB009D0B8C0B7A0B690B580B480B370B270BFB
:10990B00170B070AF70AE70AD80AC90ABA0AAA0AFA
:10991B00AA0AAA0AAA0AAA0AAA0AAA0AAA0AAA0A9C
:10992B00AA0AAA0AAA0AAA0AAA0AAA0AAA0AAA0A8C
:10993B00AA0AAA0AAA0AAA0AAA0AAA0AAA0AAA0A7C
:01994B00AA71
:011A1500FFD1
:1026DC00E4900253F0FB7A007955900258121624BC
:1026EC000000000AE4FD122ED87555011230A7E443
:1026FC00900252F0900252E0FFC39463502A75F09E
:10270C000AEFA42400F582E5F0342AAF82FE7B00A8
:10271C007A007955900259E4F0A3740AF012281D3E
:0B272C00900252E004F080CC022EB2BC
:10300B00202012301608301C0A1230AF8005D21C5B
:06301B00122989D22022D7
:102F9500901A15E493600C1226DC7E1A7F15E4FD69
:092FA500122F5CE49002A5F02259
:102EFC009002A5E075F00AA42400F9742A35F0FAC2
:102F0C007BFF78557C007D007E007F0A12152AC25B
:022F1C00202271
:102E3A001230A79002A5E075F00AA42400F582E5F5
:102E4A00F0342AAF82FE7B007A007955900259E469
:0B2E5A00F0A3740AF012281D022EB233
:061A0000122E3AC2202262
:0A1BFF00900253EDF0900252EFF057
:101C0900D39B5003021CDDE024FFFEE434FF900265
:101C190057F0A3CEF0EB14900256F0900253E02453
:101C2900FFFFE434FFFE900257E0FCA3E0FDD39FE1
:101C3900EE6480F8EC6480984003021DAE902A009F
:101C490075F00AED121655EC75F00AA42583AF82DA
:101C590090025EF0A3EFF0900256E075F00AA4241A
:101C690000F9742A35F0FA90025B74FFF0A3EAF0E8
:101C7900A3E9F0E4900259F0A3F090025BA3E475A4
:101C8900F0011215D9FEAFF090025EE475F0011271
:101C990015D985F082F583E493FD1225F290025A55
:101CA900E004F07006900259E004F0C390025AE093
:101CB900940A900259E0940040C0122EB290025842
:101CC900E004F07006900257E004F0900256E00438
:101CD900F0021C24900253E024FFFEE434FF90023A
:101CE90057F0A3CEF0900255E014A3F0900252E011
:101CF90024FFFFE434FFFE900257E0FCA3E0FDC39C
:101D09009FEE6480F8EC6480985003021DAE902A1F
:101D19000075F00AED121655EC75F00AA42583AF8B
:101D29008290025EF0A3EFF0900256E075F00AA4EB
:101D39002400F9742A35F0FA90025B74FFF0A3EAE3
:101D4900F0A3E9F0E4900259F0A3F090025BA3E458
:101D590075F0011215D9FEAFF090025EE475F0013D
:101D69001215D985F082F583E493FD1225F29002CC
:101D79005AE004F07006900259E004F0C390025A48
:101D8900E0940A900259E0940040C0122EB29002E9
:101D990058E024FFF0900257E034FFF0900256E03B
:051DA90014F0021CF51E
:011DAE002212
:051DAF00900252EDF06E
:101DB400EF14900262F0EB14A3F0900252E014FFCF
:101DC400900262E0D39F4003021F0EA3E075F00A65
:101DD400A42400F582E5F0342AAF82FEE490026484
:101DE400F0A3F0900264E0FCA3E0FDC3940AEC9439
:101DF40000502B0FEFAA0670010E14F5828A83E4BB
:101E040093FB74582DF582E43402F583EBF09002D1
:101E140065E004F070CD900264E004F080C59002A7
:101E240063E075F00AA42400F9742A35F0FA9002EC
:101E34005374FFF0A3EAF0A3E9F0900262E075F0B6
:101E44000AA42400F582E5F0342AAF82900256F009
:101E5400A3EFF0E4900264F0A3F0900253A3E475BE
:101E6400F0011215D9FEAFF0900256E475F001129C
:101E740015D985F082F583E493FD1225F29002656D
:101E8400E004F07006900264E004F0C3900265E0A0
:101E9400940A900264E0940040C0900262E075F0FD
:101EA4000AA42400F9742A35F0FA90025374FFF05E
:101EB400A3EAF0A3E9F0E4900264F0A3F0900264D2
:101EC400E0FCA3E0FDC3940AEC9400502D9002536F
:101ED400A3E475F0011215D9FEAFF074582DF58204
:101EE400E43402F583E0FD1225F2900265E004F08B
:101EF40070CB900264E004F080C3122EB2900262B0
:0A1F0400E004F0A3E004F0021DBEAB
:011F0E0022B0
:07211F00900273EBF0AC0726
:10212600A2AFE433A3F0A3E58EF0A3E589F0A3E51F
:102136008DF0A3E58BF0A28EE433A3F0AF05A3E404
:10214600F0A3EFF0E07F00FE90027AF0A3EFF0AD8F
:1021560004EDFF90027AEEF0A3EFF0900208E0FEA5
:10216600A3E0FF900204E0FCA3E0FDB507EDECB5AB
:1021760006E990020CE0FEA3E0FFEDB507DDECB545
:1021860006D920C5D6C2AF9002A5740FF01230A7AB
:102196009002A5E075F00AA42400F9742A35F0FA35
:1021A60090027C74FFF0A3EAF0A3E9F0E4A3F090B8
:1021B600027AE0FCA3E0FFECFD900273E0FBE49002
:1021C60002A4F0D224122301900280EFF0FD9002C7
:1021D6007CA3E475F0011215D9FEAFF01225F2903A
:1021E600027BE004F0700690027AE004F090027F31
:1021F600E004F0E0C3940A40B6122EB29002A5E0C5
:1022060004F0E0C3941E40851228A2900274E024D4
:06221600FF92AF0230C58B
:07201700900281EBF0AC0721
:10201E00A2AFE433A3F0A3E58EF0A3E589F0A3E528
:10202E008DF0A3E58BF0A28EE433A3F0AF05900202
:10203E008AE4F0A3EFF0E07F00FE90028AF0A3EFB7
:10204E00F0AD04EDFF90028AEEF0A3EFF0900208DF
:10205E00E0FEA3E0FF900204E0FCA3E0FDB507ED77
:10206E00ECB506E990020CE0FEA3E0FFEDB507DD4E
:10207E00ECB506D920C5D6C2AF9002A5740FF0906C
:10208E0002A5E0FFC3941E507A75F00AEFA4240057
:10209E00F582E5F0342AAF8290028CF0A3EFF0E4E3
:1020AE00900288F0A3F090028AE0FCA3E0FFECFD22
:1020BE00900281E0FB90028CE475F0011215D98537
:1020CE00F082F583E4939002A4F0C22412230190CF
:1020DE00028BE004F0700690028AE004F090028910
:1020EE00E004F07006900288E004F0C3900289E0EC
:1020FE00940A900288E0940040AC9002A5E004F0AF
:10210E0002208D1228A2900282E024FF92AF0230AC
:01211E00C5FB
:052ED800900257EDF02F
:102EDD0090025874FF1215F1EC4D4E4F6010900298
:0E2EED0057E0121569740129F9E43AFA80E2FF
:012EFB0022B4
:102FDE00E4FD0FEFAA0670010E14F5828A83E060FD
:062FEE00030D80EEAF05AB
:012FF40022BA
:1027370090028EEBF0A3EAF0A3E9F090029474FF05
:10274700F5F01215D945F06034900291E0FBA3E053
:10275700FAA3E0F9121550FF90028EE0FBA3E0FA0E
:10276700A3E0F9EF12156990028FE475F0011215D5
:0E277700C3900292E475F0011215C380BE22D9
:042F79008F828E8332
:102F7D00A2AF9226C2AF75B681758F03E4F0F58FBF
:072F8D0075B680A22692AF89
:012F9400221A
:042F5C008F828E834F
:102F6000A2AF9226C2AF758F0175B681EDF075B62E
:082F700080E4F58FA22692AF68
:012F78002236
:1027D10090026CEEF0A3EFF0A3ECF0A3EDF0EB4A66
:1027E100603990026CE0FEA3E0FFA3E0FCA3E0F5FA
:1027F100828C83E0FD122F5CEB1B70011A90026F3B
:10280100E004F0700690026EE004F090026DE004C6
:0C281100F070CB90026CE004F080C32259
:0830A700E4900000F0A3F02208
:102EB200900000E0FEA3E0FF122F79900000E0FEF8
:102EC200A3E0FF7C007D027B007A021227D1E4900E
:062ED2000000F0A3F02255
:0A25F200A905900266EEF0A3EFF0D9
:1025FC00EE54FEFE900000E0FCA3E0FD7002EE6CD9
:10260C006059ED4C6003122EB2900266E0FEEE545F
:10261C00FEFE7F00900000F0A3EFF0900268EEF059
:10262C00A3EFF0A37400F0A37402F07F007E02907D
:10263C000268E475F0011215D985F082F583E493F4
:10264C00FD90026AE475F0011215D985F082F583CC
:10265C00EDF0EF1F70011EEF4E70D4900266E0FC9F
:10266C00A3E0FDEC5401FC74022DF58274003CF5E2
:03267C0083E9F0FF
:01267F002238
:10281D00900254EEF0A3EFF0A3EBF0A3EAF0A3E9DE
:10282D00F090025974FFF5F01215D945F06026901D
:10283D000254E475F0011215D9AFF0FE900256E086
:10284D00FBA3E475F0011215D9A9F0FA121550FD8C
:06285D001225F280CC22DE
:102F1E00900270EFF0A3EDF07F0A12254990027037
:102F2E00E0FF122549900271E0FF1225490230C5DB
:0830AF007F021225490230C521
:062DDE001230CCEF60276B
:102DE4009002527402F0A37496F01229BF9002521A
:102DF400E475F0011215D985F082F583EFF01230F5
:072E0400D2EF70E67F01220E
:032E0B007F002223
:10302100900252EFF07F2F122549900252E0FF12D9
:0530310025490230C535
:10303600900252EFF07F30122549900252E0FF12C3
:0530460025490230C520
:102FAE00D209D208D207D206D205D204D203D20257
:082FBE00D201E4F54FD21E22FE
:102FC600C209C208C207C206C205C204C203C202BF
:082FD600C201E4F54FD21E22F6
:0230DA00C12310
:0F304B0075C04475CFE2C2C343F60275C30122BC
:1028A2007E027F0E900206EEF0A3EFF090020AEE97
:1028B200F0A3EFF0900202EEF0A3EFF07E027F2E83
:1028C200900208EEF0A3EFF090020CEEF0A3EFF00E
:0D28D200900204EEF0A3EFF0C22202304BA2
:1029180090020AE475F0011215D985F082F583EF6B
:10292800F090020AE475F0011215D985F082F5835A
:10293800EDF090020AE0B4020FA3E0B42E0A900270
:092948000A7402F0A3740EF022DF
:0730C500C222C2C4D2C522E1
:10254900202255D22290020CE475F0011215D9858A
:10255900F082F58374FFF07C027D4E90020CE0B5A9
:10256900040FA3E0B5050A90020C7402F0A3742EBF
:10257900F090020CE475F0011215D985F082F5830B
:10258900E4F090020CE0B5040FA3E0B5050A90024F
:102599000C7402F0A3742EF090020CE475F0011291
:1025A90015D985F082F583E4F090020CE0B4020FAE
:1025B900A3E0B44E0A90020C7402F0A3742EF090BA
:1025C900020CE475F0011215D985F082F583EFF05C
:1025D90090020CE0B4020FA3E0B44E0A90020C740E
:0925E90002F0A3742EF07F012220
:102E0E00900206E0FCA3E0FD900202E0B50408A3E8
:102E1E00E0B505037F0022900206E0FCA3E0F582F8
:0C2E2E008C83E0B507037F01227F0022A7
:1029BF00900207E004F07006900206E004F0900227
:1029CF0006E475F0011215D985F082F583E0FF90CA
:1029DF000206E0B4020FA3E0B42E0A9002067402BE
:0529EF00F0A3740EF0DE
:0129F40022C0
:0630CC007FFF122E0E2210
:0630D200E4FF122E0E22A5
:031A18000216DCD7
:1016DC00C0E0C0F0C083C082C0D075D000C000C0D4
:1016EC0004C005C006C007E5C154F812166118D332
:1016FC000017370817371017851817D12017DE2851
:10170C00186930187538188650188658189960184A
:10171C00886818997018887818868018A888188690
:10172C009018A89818BBA000001900C2C59002051B
:10173C00E004F07006900204E004F07E027F4E900C
:10174C000204E0B5060FA3E0B5070A900204740288
:10175C00F0A3742EF0900204E475F0011215D985F3
:10176C00F082F583E0F5C2900204E06E7003A3E012
:10177C006F600302190002185C900205E004F0701F
:10178C0006900204E004F07E027F4E900204E0B565
:10179C00060FA3E0B5070A9002047402F0A3742E9E
:1017AC00F0900204E475F0011215D985F082F583EE
:1017BC00E0F5C2900204E06E7003A3E06F600302D8
:1017CC00190002185C900208E0FFA3E0900204CF1D
:1017DC00801B90020CE0FEA3E0FF900204E0FCA34F
:1017EC00E0FDB50713ECB5060F900208EEF0A3EF81
:1017FC00F0C2C5D2C40219008D828C83E0B4FF07FD
:10180C00C2C4D2C5021900900205E004F070069023
:10181C000204E004F07E027F4E900204E0B5060F55
:10182C00A3E0B5070A9002047402F0A3742EF090A2
:10183C000204E475F0011215D985F082F583E0F508
:10184C00C2900204E06E7003A3E06F600302190003
:10185C009002047402F0A3742EF002190090020896
:10186C00E0FFA3E0900204803D900208E0FFA3E0BB
:10187C00900204CFF0A3EFF0807A8017900208E07A
:10188C00FFA3E0900204CFF0A3EFF0D223ADC27F10
:10189C00FF8004ADC2E4FF1229188058900202E0C8
:1018AC00FFA3E090020ACFF0A3EFF0D2C4804590E2
:1018BC00020AE0FFA3E0900202CFF0A3EFF0302386
:1018CC0033D2C5C223802D900208E0FEA3E0FF9026
:1018DC000204EEF0A3EFF0900202E0FDA3E0900210
:1018EC000ACDF0A3EDF0D2C4A3E06E7003A3E06FB9
:1018FC006002D2C5C2C3D007D006D005D004D00038
:0B190C00D0D0D082D083D0F0D0E032E9
:072301009002A1EFF0A90515
:10230800C22520C3FD20C5FAC2C4D2C5E4FFFD30F2
:10231800C3FD30C3FDE5C154F8FC64086004ECB4A7
:102328001013EFB40105EB44018003EB54FEF5C232
:102338007D010223CDECB4180B89C27D02C2C4C250
:10234800C50223CDECB420028045EC6428703CED36
:10235800B4020E9002A1E0F5C27D03C2C5C2C480DA
:1023680064EDB4031B302408D2C57F01C2C4805574
:102378009002A4E0F5C2C2C57D04E4FFC2C4804552
:10238800ED64047040D2C47D05803AECB4300AD2C2
:10239800C4D2C57D08E4FF802CECB438028022EC5E
:1023A800B44006C2C2C2C5801CECB448028012EC1C
:1023B800B450028004ECB45808D2C47D07AEC28081
:1023C80004D2C4D2C5C2C3ED64076008ED640560D9
:0623D8000302231AAF0608
:0123DE0022DC
:100A1A00020A9AE493A3F8E493A34003F68001F24E
:100A2A0008DFF48029E493A3F85407240CC8C333DD
:100A3A00C4540F4420C8834004F456800146F6DFAC
:100A4A00E4800B01020408102040809030D8E47E34
:100A5A00019360BCA3FF543F30E509541FFEE493A1
:100A6A00A360010ECF54C025E060A840B8E493A368
:100A7A00FAE493A3F8E493A3C8C582C8CAC583CA93
:100A8A00F0A3C8C582C8CAC583CADFE9DEE780BE4B
:0130DC0000F3
:10145A00E709F608DFFA8046E709F208DFFA803E74
:10146A0088828C83E709F0A3DFFA8032E309F60861
:10147A00DFFA8078E309F208DFFA807088828C83C9
:10148A00E309F0A3DFFA806489828A83E0A3F6087D
:10149A00DFFA805889828A83E0A3F208DFFA804C57
:1014AA0080D280FA80C680D4806980F2803380102E
:1014BA0080A680EA809A80A880DA80E280CA803397
:1014CA0089828A83ECFAE493A3C8C582C8CCC5830F
:1014DA00CCF0A3C8C582C8CCC583CCDFE9DEE780DF
:1014EA000D89828A83E493A3F608DFF9ECFAA9F05E
:1014FA00EDFB2289828A83ECFAE0A3C8C582C8CCB4
:10150A00C583CCF0A3C8C582C8CCC583CCDFEADECC
:10151A00E880DB89828A83E493A3F208DFF980CC2E
:10152A0088F0EF60010E4E60C388F0ED2402B40427
:10153A000050B9F582EB2402B4040050AF232345CE
:06154A0082239014AA7335
:10155000BB010689828A83E0225002E722BBFE0299
:09156000E32289828A83E49322CC
:10156900BB010689828A83F0225002F722BBFE0161
:02157900F3225B
:10157B00EF8DF0A4A8F0CF8CF0A428CE8DF0A42E84
:02158B00FE223E
:10158D00C2D5EC30E709B2D5E4C39DFDE49CFCEE79
:10159D0030E715B2D5E4C39FFFE49EFE121687C354
:1015AD00E49DFDE49CFC800312168730D507C3E44F
:0615BD009FFFE49EFE22E8
:1015C300C5F0F8A3E028F0C5F0F8E58215827002B3
:0615D3001583E038F02250
:1015D900A3F8E0C5F025F0F0E582158270021583C5
:0615E900E0C838F0E82222
:1015EF007401FF3395E0FEFDFCA3A3A3E0CF2FF022
:1015FF00E582158270021583E0CE3EF0E5821582FA
:10160F0070021583E0CD3DF0E582158270021583DF
:05161F00E0CC3CF022CC
:10162400A8828583F0D083D08212163B12163B1217
:10163400163B12163BE473E493A3C583C5F0C5833C
:10164400C8C582C8F0A3C583C5F0C583C8C582C810
:011654002273
:0C165500A42582F582E5F03583F58322A0
:10166100D083D082F8E4937012740193700DA3A318
:1016710093F8740193F5828883E47374029368602C
:06168100EFA3A3A380DF2C
:10168700BC000BBE0029EF8DF084FFADF022E4CC47
:10169700F875F008EF2FFFEE33FEEC33FCEE9DEC10
:1016A700984005FCEE9DFE0FD5F0E9E4CEFD22ED56
:1016B700F8F5F0EE8420D21CFEADF075F008EF2FA0
:1016C700FFED33FD4007985006D5F0F222C398FD91
:0516D7000FD5F0EA222E
:00000001FF
